 FEC

 Timestamp is 4da293c9 (Mon Apr 11 17:38:17 2011)

 Preferred load address is 10000000

 Start         Length     Name                   Class
 0001:00000000 00000004H .CRT$XCA                CODE
 0001:00000004 00000004H .CRT$XCZ                CODE
 0001:00000008 00000004H .CRT$XIA                CODE
 0001:0000000c 00000004H .CRT$XIZ                CODE
 0001:00000010 00000004H .CRT$XPA                CODE
 0001:00000014 00000004H .CRT$XPZ                CODE
 0001:00000018 00000004H .CRT$XTA                CODE
 0001:0000001c 00000004H .CRT$XTZ                CODE
 0001:00000020 00000084H .rdata                  CODE
 0001:000000a4 00000020H .rdata$debug            CODE
 0001:000000c4 00002ac4H .text                   CODE
 0001:00002b88 0000001cH .xdata                  CODE
 0001:00002ba4 00000050H .idata$2                CODE
 0001:00002bf4 00000014H .idata$3                CODE
 0001:00002c08 000000b8H .idata$4                CODE
 0001:00002cc0 00000298H .idata$6                CODE
 0001:00002f60 00000046H .edata                  CODE
 0002:00000000 000000b8H .idata$5                DATA
 0002:000000b8 00000b14H .data                   DATA
 0002:00000be0 00000160H .bss                    DATA
 0003:00000000 000001f0H .pdata                  DATA

  Address         Publics by Value              Rva+Base       Lib:Object

 0000:00000000       ___safe_se_handler_count   00000000     <absolute>
 0000:00000000       ___safe_se_handler_table   00000000     <absolute>
 0001:00000000       __xc_a                     10001000     corelib0:crt0init.obj
 0001:00000004       __xc_z                     10001004     corelib0:crt0init.obj
 0001:00000008       __xi_a                     10001008     corelib0:crt0init.obj
 0001:0000000c       __xi_z                     1000100c     corelib0:crt0init.obj
 0001:00000010       __xp_a                     10001010     corelib0:crt0init.obj
 0001:00000014       __xp_z                     10001014     corelib0:crt0init.obj
 0001:00000018       __xt_a                     10001018     corelib0:crt0init.obj
 0001:0000001c       __xt_z                     1000101c     corelib0:crt0init.obj
 0001:0000003c       ??_C@_0CA@LDJKLMPP@Freescale?5Fast?5Ethernet?5Adapter?$AA@ 1000103c     fec_common_topaz_v1:fec.obj
 0001:0000005c       ??_C@_1BI@DCGEADED@?$AAM?$AAA?$AAC?$AAA?$AAd?$AAd?$AAr?$AAe?$AAs?$AAs?$AA1?$AA?$AA@ 1000105c     fec_common_topaz_v1:fec.obj
 0001:00000074       ??_C@_1BI@CANBKMKN@?$AAM?$AAA?$AAC?$AAA?$AAd?$AAd?$AAr?$AAe?$AAs?$AAs?$AA2?$AA?$AA@ 10001074     fec_common_topaz_v1:fec.obj
 0001:0000008c       ??_C@_1BI@JIGNMLMI@?$AAM?$AAA?$AAC?$AAA?$AAd?$AAd?$AAr?$AAe?$AAs?$AAs?$AA3?$AA?$AA@ 1000108c     fec_common_topaz_v1:fec.obj
 0001:000000c4       BSPFECPowerEnable          100010c4 f   bspfec.obj
 0001:000000c8       BSPFECClockConfig          100010c8 f   bspfec.obj
 0001:00000124       BSPFECGetIrq               10001124 f   bspfec.obj
 0001:0000012c       BSPFECBaseAddress          1000112c f   bspfec.obj
 0001:00000138       BSPFECusesRMII             10001138 f   bspfec.obj
 0001:00000140       BSPPhyReset                10001140 f   bspfec.obj
 0001:0000039c       BSPFECIomuxConfig          1000139c f   bspfec.obj
 0001:000003b4       GetMacAddFromUUID          100013b4 f   fec_common_topaz_v1:fec.obj
 0001:0000049c       FECSetPower                1000149c f   fec_common_topaz_v1:fec.obj
 0001:00000504       FECHalt                    10001504 f   fec_common_topaz_v1:fec.obj
 0001:00000588       FECQueryInformation        10001588 f   fec_common_topaz_v1:fec.obj
 0001:000008c8       FECReset                   100018c8 f   fec_common_topaz_v1:fec.obj
 0001:00000960       FECSend                    10001960 f   fec_common_topaz_v1:fec.obj
 0001:00000a10       FECTransferData            10001a10 f   fec_common_topaz_v1:fec.obj
 0001:00000b18       FECSetInformation          10001b18 f   fec_common_topaz_v1:fec.obj
 0001:00000d7c       FECShutdown                10001d7c f   fec_common_topaz_v1:fec.obj
 0001:00000da8       FECCheckForHang            10001da8 f   fec_common_topaz_v1:fec.obj
 0001:000011f0       DriverEntry                100021f0 f   fec_common_topaz_v1:fec.obj
 0001:000012fc       FECIsr                     100022fc f   fec_common_topaz_v1:interrupt.obj
 0001:0000130c       FECDisableInterrupt        1000230c f   fec_common_topaz_v1:interrupt.obj
 0001:0000132c       FECEnableInterrupt         1000232c f   fec_common_topaz_v1:interrupt.obj
 0001:0000134c       ProcessReceiveInterrupts   1000234c f   fec_common_topaz_v1:interrupt.obj
 0001:0000152c       ProcessTransmitInterrupts  1000252c f   fec_common_topaz_v1:interrupt.obj
 0001:000016c0       ProcessMIIInterrupts       100026c0 f   fec_common_topaz_v1:interrupt.obj
 0001:00001730       FECHandleInterrupt         10002730 f   fec_common_topaz_v1:interrupt.obj
 0001:000017d8       FECStartXmit               100027d8 f   fec_common_topaz_v1:chip.obj
 0001:0000191c       FECQueueMII                1000291c f   fec_common_topaz_v1:chip.obj
 0001:00001994       FECDoMIICmd                10002994 f   fec_common_topaz_v1:chip.obj
 0001:000019e0       FECParseMIISr              100029e0 f   fec_common_topaz_v1:chip.obj
 0001:00001a08       FECParseMIICr              10002a08 f   fec_common_topaz_v1:chip.obj
 0001:00001a28       FECParseMIIAnar            10002a28 f   fec_common_topaz_v1:chip.obj
 0001:00001a58       FECParseAm79c874Dr         10002a58 f   fec_common_topaz_v1:chip.obj
 0001:00001ab4       FECParseKSZ8041NLPC2       10002ab4 f   fec_common_topaz_v1:chip.obj
 0001:00001b28       FECParseLAN8700SCSR        10002b28 f   fec_common_topaz_v1:chip.obj
 0001:00001b88       FECParseDP83640PHYSTS      10002b88 f   fec_common_topaz_v1:chip.obj
 0001:00001be8       FECParsePHYLink            10002be8 f   fec_common_topaz_v1:chip.obj
 0001:00001cc0       FECGetPHYId2               10002cc0 f   fec_common_topaz_v1:chip.obj
 0001:00001d38       FECGetLinkStatus           10002d38 f   fec_common_topaz_v1:chip.obj
 0001:00001d64       FECDispPHYCfg              10002d64 f   fec_common_topaz_v1:chip.obj
 0001:00001d70       FECEnetDeinit              10002d70 f   fec_common_topaz_v1:chip.obj
 0001:00001e18       FECEnetAutoNego            10002e18 f   fec_common_topaz_v1:chip.obj
 0001:00001e74       FECEnetPowerHandle         10002e74 f   fec_common_topaz_v1:chip.obj
 0001:00001eb0       FECEnetReset               10002eb0 f   fec_common_topaz_v1:chip.obj
 0001:00002078       CalculateHashValue         10003078 f   fec_common_topaz_v1:chip.obj
 0001:000020c4       AddMultiCast               100030c4 f   fec_common_topaz_v1:chip.obj
 0001:0000210c       ClearAllMultiCast          1000310c f   fec_common_topaz_v1:chip.obj
 0001:0000213c       FECGetPHYId                1000313c f   fec_common_topaz_v1:chip.obj
 0001:000021e0       FECEnetInit                100031e0 f   fec_common_topaz_v1:chip.obj
 0001:00002550       NdisMSleep                 10003550 f   ndis:NDIS.dll
 0001:00002560       NdisFreeMemory             10003560 f   ndis:NDIS.dll
 0001:00002570       NdisMDeregisterIoPortRange 10003570 f   ndis:NDIS.dll
 0001:00002580       NdisMDeregisterInterrupt   10003580 f   ndis:NDIS.dll
 0001:00002590       NdisMDeregisterAdapterShutdownHandler 10003590 f   ndis:NDIS.dll
 0001:000025a0       NdisQueryPacket            100035a0 f   ndis:NDIS.dll
 0001:000025b0       NdisCloseConfiguration     100035b0 f   ndis:NDIS.dll
 0001:000025c0       NdisWriteErrorLogEntry     100035c0 f   ndis:NDIS.dll
 0001:000025d0       NdisMRegisterInterrupt     100035d0 f   ndis:NDIS.dll
 0001:000025e0       NdisMRegisterAdapterShutdownHandler 100035e0 f   ndis:NDIS.dll
 0001:000025f0       NdisMRegisterIoPortRange   100035f0 f   ndis:NDIS.dll
 0001:00002600       NdisReadConfiguration      10003600 f   ndis:NDIS.dll
 0001:00002610       NdisOpenConfiguration      10003610 f   ndis:NDIS.dll
 0001:00002620       NdisMSetAttributesEx       10003620 f   ndis:NDIS.dll
 0001:00002630       NdisAllocateMemory         10003630 f   ndis:NDIS.dll
 0001:00002640       NdisTerminateWrapper       10003640 f   ndis:NDIS.dll
 0001:00002650       NdisMRegisterMiniport      10003650 f   ndis:NDIS.dll
 0001:00002660       NdisInitializeWrapper      10003660 f   ndis:NDIS.dll
 0001:00002670       NdisMIndicateStatusComplete 10003670 f   ndis:NDIS.dll
 0001:00002680       NdisMIndicateStatus        10003680 f   ndis:NDIS.dll
 0001:00002690       Sleep                      10003690 f   coredll:COREDLL.dll
 0001:000026a0       DisableThreadLibraryCalls  100036a0 f   coredll:COREDLL.dll
 0001:000026b0       KernelIoControl            100036b0 f   coredll:COREDLL.dll
 0001:000026c0       LeaveCriticalSection       100036c0 f   coredll:COREDLL.dll
 0001:000026d0       EnterCriticalSection       100036d0 f   coredll:COREDLL.dll
 0001:000026e0       DeleteCriticalSection      100036e0 f   coredll:COREDLL.dll
 0001:000026f0       InitializeCriticalSection  100036f0 f   coredll:COREDLL.dll
 0001:00002700       HalFreeCommonBuffer        10003700 f   ceddk:CEDDK.dll
 0001:00002710       HalAllocateCommonBuffer    10003710 f   ceddk:CEDDK.dll
 0001:00002720       DDKClockSetGatingMode      10003720 f   cspddk:CSPDDK.dll
 0001:00002730       DDKGpioWriteDataPin        10003730 f   cspddk:CSPDDK.dll
 0001:00002740       DDKGpioSetConfig           10003740 f   cspddk:CSPDDK.dll
 0001:00002750       DDKIomuxSetPadConfig       10003750 f   cspddk:CSPDDK.dll
 0001:00002760       DDKIomuxSetPinMux          10003760 f   cspddk:CSPDDK.dll
 0001:00002770       DllMain                    10003770 f   corelib0:dllmain.obj
 0001:0000287c       _DllMainCRTStartup         1000387c f   corelib0:pegdmain.obj
 0001:000028a8       __GSHandlerCheckCommon     100038a8 f   corelib0:gshandler.obj
 0001:000028e0       __GSHandlerCheck           100038e0 f   corelib0:gshandler.obj
 0001:00002900       __security_init_cookie     10003900 f   corelib0:seccinit.obj
 0001:0000294c       __security_check_cookie    1000394c f   corelib0:armsecgs.obj
 0001:0000295c       __gsfailure                1000395c     corelib0:armsecgs.obj
 0001:00002a60       _cexit                     10003a60 f   corelib0:cexit.obj
 0001:00002a70       _initterm                  10003a70 f   corelib0:crt0dat.obj
 0001:00002a9c       _cinit                     10003a9c f   corelib0:crt0dat.obj
 0001:00002afc       __crt_ExitProcess          10003afc f   corelib0:exitproc_proxy.obj
 0001:00002b08       memcpy                     10003b08 f   corelib1:COREDLL.dll
 0001:00002b18       memset                     10003b18 f   corelib1:COREDLL.dll
 0001:00002b28       _XcptFilter                10003b28 f   corelib1:COREDLL.dll
 0001:00002b38       __C_specific_handler       10003b38 f   corelib1:COREDLL.dll
 0001:00002b48       __security_gen_cookie2     10003b48 f   corelib1:COREDLL.dll
 0001:00002b58       __report_gsfailure         10003b58 f   corelib1:COREDLL.dll
 0001:00002b68       free                       10003b68 f   corelib1:COREDLL.dll
 0001:00002b78       TerminateProcess           10003b78 f   coredll:COREDLL.dll
 0001:00002ba4       __IMPORT_DESCRIPTOR_NDIS   10003ba4     ndis:NDIS.dll
 0001:00002bb8       __IMPORT_DESCRIPTOR_COREDLL 10003bb8     coredll:COREDLL.dll
 0001:00002bcc       __IMPORT_DESCRIPTOR_CEDDK  10003bcc     ceddk:CEDDK.dll
 0001:00002be0       __IMPORT_DESCRIPTOR_CSPDDK 10003be0     cspddk:CSPDDK.dll
 0001:00002bf4       __NULL_IMPORT_DESCRIPTOR   10003bf4     ndis:NDIS.dll
 0002:00000000       __imp_HalFreeCommonBuffer  10004000     ceddk:CEDDK.dll
 0002:00000004       __imp_HalAllocateCommonBuffer 10004004     ceddk:CEDDK.dll
 0002:00000008       \177CEDDK_NULL_THUNK_DATA  10004008     ceddk:CEDDK.dll
 0002:0000000c       __imp_free                 1000400c     corelib1:COREDLL.dll
 0002:00000010       __imp___report_gsfailure   10004010     corelib1:COREDLL.dll
 0002:00000014       __imp___C_specific_handler 10004014     corelib1:COREDLL.dll
 0002:00000018       __imp__XcptFilter          10004018     corelib1:COREDLL.dll
 0002:0000001c       __imp_memset               1000401c     corelib1:COREDLL.dll
 0002:00000020       __imp_memcpy               10004020     corelib1:COREDLL.dll
 0002:00000024       __imp___security_gen_cookie2 10004024     corelib1:COREDLL.dll
 0002:00000028       __imp_LeaveCriticalSection 10004028     coredll:COREDLL.dll
 0002:0000002c       __imp_InitializeCriticalSection 1000402c     coredll:COREDLL.dll
 0002:00000030       __imp_DeleteCriticalSection 10004030     coredll:COREDLL.dll
 0002:00000034       __imp_EnterCriticalSection 10004034     coredll:COREDLL.dll
 0002:00000038       __imp_TerminateProcess     10004038     coredll:COREDLL.dll
 0002:0000003c       __imp_KernelIoControl      1000403c     coredll:COREDLL.dll
 0002:00000040       __imp_DisableThreadLibraryCalls 10004040     coredll:COREDLL.dll
 0002:00000044       __imp_Sleep                10004044     coredll:COREDLL.dll
 0002:00000048       \177COREDLL_NULL_THUNK_DATA 10004048     coredll:COREDLL.dll
 0002:0000004c       __imp_DDKIomuxSetPadConfig 1000404c     cspddk:CSPDDK.dll
 0002:00000050       __imp_DDKIomuxSetPinMux    10004050     cspddk:CSPDDK.dll
 0002:00000054       __imp_DDKGpioSetConfig     10004054     cspddk:CSPDDK.dll
 0002:00000058       __imp_DDKGpioWriteDataPin  10004058     cspddk:CSPDDK.dll
 0002:0000005c       __imp_DDKClockSetGatingMode 1000405c     cspddk:CSPDDK.dll
 0002:00000060       \177CSPDDK_NULL_THUNK_DATA 10004060     cspddk:CSPDDK.dll
 0002:00000064       __imp_NdisAllocateMemory   10004064     ndis:NDIS.dll
 0002:00000068       __imp_NdisMSetAttributesEx 10004068     ndis:NDIS.dll
 0002:0000006c       __imp_NdisTerminateWrapper 1000406c     ndis:NDIS.dll
 0002:00000070       __imp_NdisReadConfiguration 10004070     ndis:NDIS.dll
 0002:00000074       __imp_NdisMRegisterMiniport 10004074     ndis:NDIS.dll
 0002:00000078       __imp_NdisInitializeWrapper 10004078     ndis:NDIS.dll
 0002:0000007c       __imp_NdisMIndicateStatusComplete 1000407c     ndis:NDIS.dll
 0002:00000080       __imp_NdisMIndicateStatus  10004080     ndis:NDIS.dll
 0002:00000084       __imp_NdisOpenConfiguration 10004084     ndis:NDIS.dll
 0002:00000088       __imp_NdisMRegisterIoPortRange 10004088     ndis:NDIS.dll
 0002:0000008c       __imp_NdisMRegisterAdapterShutdownHandler 1000408c     ndis:NDIS.dll
 0002:00000090       __imp_NdisMRegisterInterrupt 10004090     ndis:NDIS.dll
 0002:00000094       __imp_NdisWriteErrorLogEntry 10004094     ndis:NDIS.dll
 0002:00000098       __imp_NdisCloseConfiguration 10004098     ndis:NDIS.dll
 0002:0000009c       __imp_NdisQueryPacket      1000409c     ndis:NDIS.dll
 0002:000000a0       __imp_NdisMDeregisterAdapterShutdownHandler 100040a0     ndis:NDIS.dll
 0002:000000a4       __imp_NdisMDeregisterInterrupt 100040a4     ndis:NDIS.dll
 0002:000000a8       __imp_NdisMDeregisterIoPortRange 100040a8     ndis:NDIS.dll
 0002:000000ac       __imp_NdisFreeMemory       100040ac     ndis:NDIS.dll
 0002:000000b0       __imp_NdisMSleep           100040b0     ndis:NDIS.dll
 0002:000000b4       \177NDIS_NULL_THUNK_DATA   100040b4     ndis:NDIS.dll
 0002:00000160       Am79c874Config             10004160     fec_common_topaz_v1:chip.obj
 0002:00000180       Am79c874Startup            10004180     fec_common_topaz_v1:chip.obj
 0002:000001a0       Am79c874Ackint             100041a0     fec_common_topaz_v1:chip.obj
 0002:000001c0       Am79c874Shutdown           100041c0     fec_common_topaz_v1:chip.obj
 0002:000001d0       Am79c874Info               100041d0     fec_common_topaz_v1:chip.obj
 0002:000003e4       LAN8700Config              100043e4     fec_common_topaz_v1:chip.obj
 0002:00000404       LAN8700Startup             10004404     fec_common_topaz_v1:chip.obj
 0002:00000424       LAN8700Ackint              10004424     fec_common_topaz_v1:chip.obj
 0002:0000043c       LAN8700Shutdown            1000443c     fec_common_topaz_v1:chip.obj
 0002:0000044c       PhyInfo                    1000444c     fec_common_topaz_v1:chip.obj
 0002:00000460       LAN8700Info                10004460     fec_common_topaz_v1:chip.obj
 0002:00000674       DP83640Config              10004674     fec_common_topaz_v1:chip.obj
 0002:00000694       DP83640Startup             10004694     fec_common_topaz_v1:chip.obj
 0002:000006b4       DP83640Ackint              100046b4     fec_common_topaz_v1:chip.obj
 0002:000006cc       DP83640Shutdown            100046cc     fec_common_topaz_v1:chip.obj
 0002:000006e0       DP83640Info                100046e0     fec_common_topaz_v1:chip.obj
 0002:000008f4       PHYCmdCfg                  100048f4     fec_common_topaz_v1:chip.obj
 0002:00000904       PHYCmdLink                 10004904     fec_common_topaz_v1:chip.obj
 0002:00000914       PHYCmdSuspend              10004914     fec_common_topaz_v1:chip.obj
 0002:00000924       PHYCmdResume               10004924     fec_common_topaz_v1:chip.obj
 0002:00000934       KSZ8041NLConfig            10004934     fec_common_topaz_v1:chip.obj
 0002:0000095c       KSZ8041NLStartup           1000495c     fec_common_topaz_v1:chip.obj
 0002:0000097c       KSZ8041NLAckint            1000497c     fec_common_topaz_v1:chip.obj
 0002:0000099c       KSZ8041NLShutdown          1000499c     fec_common_topaz_v1:chip.obj
 0002:000009b0       KSZ8041NLInfo              100049b0     fec_common_topaz_v1:chip.obj
 0002:00000bc4       __security_cookie          10004bc4     corelib0:seccinit.obj
 0002:00000bc8       __security_cookie_complement 10004bc8     corelib0:seccinit.obj
 0002:00000be0       gpFECReg                   10004be0     fec_common_topaz_v1:fec.obj
 0002:00000be4       gMIIFree                   10004be4     fec_common_topaz_v1:chip.obj
 0002:00000be8       gMIIHead                   10004be8     fec_common_topaz_v1:chip.obj
 0002:00000bec       gMIITail                   10004bec     fec_common_topaz_v1:chip.obj
 0002:00000bf0       _exitflag                  10004bf0     corelib0:cexit.obj
 0002:00000c00       gMIICmds                   10004c00     <common>
 0002:00000cf0       gFECNdisHandle             10004cf0     <common>
 0002:00000d00       gFECBufCs                  10004d00     <common>
 0002:00000d20       gFECRegCs                  10004d20     <common>
 0002:00000d34       __onexitend                10004d34     <common>
 0002:00000d38       __onexitbegin              10004d38     <common>
 0002:00000d3c       _pRawDllMain               10004d3c     <common>

 entry point at        0001:0000287c

 Static symbols

 0001:00000dc8       FECInitialize              10001dc8 f   fec_common_topaz_v1:fec.obj
 0001:0000278c       _DllMainCRTStartupHelper   1000378c f   corelib0:pegdmain.obj
 0001:000029a0       doexit                     100039a0 f   corelib0:cexit.obj
